:020000040800F2
:1000000000280020550400089904000899040008FD
:1000100099040008990400089904000800000000F1
:10002000000000000000000000000000990400082B
:10003000990400080000000099040008F10300087A
:10004000990400089904000899040008990400081C
:10005000990400089904000899040008990400080C
:1000600099040008990400089904000899040008FC
:1000700099040008990400089904000899040008EC
:1000800099040008990400089904000899040008DC
:1000900099040008990400089904000899040008CC
:1000A00099040008990400089904000899040008BC
:1000B0009904000899040008000000009904000851
:1000C00099040008000000000000000099040008E6
:1000D00000000000990400089904000800000000D6
:1000E0009904000899040008990400080000000021
:1000F0000000000000000000000000000000000000
:0C01000000000000000000005FF808F1A3
:10010C0080B483B000AF03463960FB7197F90730B8
:10011C00002B0BDA0D49FB7903F00F03043B3A6813
:10012C00D2B21201D2B20B441A7609E0084997F9FF
:10013C0007303A68D2B21201D2B20B4483F80023D2
:10014C0000BF0C37BD4680BC704700BF00ED00E01F
:10015C0000E100E080B582B000AF78607B68B3F15D
:10016C00807F01D3012311E00A4A7B6823F07F438F
:10017C00013B53600F214FF0FF30FFF7C1FF054BE0
:10018C0000229A60034B07221A6000231846083796
:10019C00BD4680BD10E000E080B500AF154A154BA0
:1001AC001B6843F0010313601249124B5A68124B3F
:1001BC0013404B600F4A0F4B1B6823F0847323F4DE
:1001CC00803313600B4A0B4B1B6823F480231360A2
:1001DC00084A084B5B6823F4FE035360054B4FF44D
:1001EC001F029A6000F078F8044B4FF000629A609E
:1001FC0000BF80BD001002400000FFF800ED00E0E1
:10020C0080B485B000AF0023FB600023BB600023EB
:10021C007B602C4B5B6803F00C03FB60FB68042BCE
:10022C0007D0082B09D0002B33D1274B274A1A6053
:10023C0033E0254B254A1A602FE0224B5B6803F410
:10024C007013BB601F4B5B6803F480337B60BB682F
:10025C009B0C0233BB607B68002B06D1BB681C4A2D
:10026C0002FB03F3184A136017E0164B5B6803F4A8
:10027C000033002B06D0BB68154A02FB03F3124A6D
:10028C0013600AE0BB68114A02FB03F30E4A1360C9
:10029C0003E00D4B0D4A1A6000BF0A4B5B6803F07C
:1002AC00F0031B090B4AD35CDBB2FB60064B1A68EC
:1002BC00FB6822FA03F3044A136000BF1437BD46EF
:1002CC0080BC7047001002400000002000127A0031
:1002DC0000093D000400002080B500AF00F002F8DA
:1002EC0000BF80BD80B483B000AF00237B600023CF
:1002FC003B603A4A394B1B6843F480331360374BED
:10030C001B6803F400333B607B6801337B603B6804
:10031C00002B03D17B68B3F5A06FF0D12F4B1B687A
:10032C0003F40033002B02D001233B6001E00023D7
:10033C003B603B68012B4BD1294A294B1B6843F08E
:10034C0010031360264A264B1B6823F0030313602B
:10035C00234A234B1B6843F0020313601F4A1F4BB5
:10036C005B6853601D4A1D4B5B6853601B4A1B4BFB
:10037C005B6843F480635360184A184B5B6823F442
:10038C007C135360154A154B5B6843F4E8135360B8
:10039C00124A124B1B6843F08073136000BF0F4B63
:1003AC001B6803F00073002BF9D00C4A0B4B5B68F5
:1003BC0023F003035360094A084B5B6843F00203C4
:1003CC00536000BF054B5B6803F00C03082BF9D19D
:1003DC0000BF0C37BD4680BC704700BF0010024008
:1003EC000020024080B400AF044B1B680133034A69
:1003FC00136000BFBD4680BC704700BF14000020D6
:10040C0080B500AFFFF7FCFE074B1B68074AA2FB49
:10041C0003235B0B1846FFF79DFE034B1B681A4624
:10042C00034B1A60F9E700BF000000205917B7D141
:10043C00180000209C04000800000020140000207C
:10044C00140000201C000020002103E00A4B5B5824
:10045C004350043109480A4B42189A42F6D3094AD0
:10046C0002E0002342F8043B074B9A42F9D3FFF712
:10047C0093FEFFF7C5FF70479C04000800000020A6
:10048C0014000020140000201C000020FEE70000D7
:10049C0000A24A0400000000000000000102030456
:0404AC00060708092E
:040000050800045596
:00000001FF
